BL51 BANKED LINKER/LOCATER V6.00                                                        09/05/2017  17:55:54  PAGE 1


BL51 BANKED LINKER/LOCATER V6.00, INVOKED BY:
C:\KEIL_UV3\C51\BIN\BL51.EXE main.obj TO MA82G5Dxx RAMSIZE (256)


MEMORY MODEL: SMALL


INPUT MODULES INCLUDED:
  main.obj (MAIN)
  C:\KEIL_UV3\C51\LIB\C51S.LIB (?C_STARTUP)


LINK MAP OF MODULE:  MA82G5Dxx (MAIN)


            TYPE    BASE      LENGTH    RELOCATION   SEGMENT NAME
            -----------------------------------------------------

            * * * * * * *   D A T A   M E M O R Y   * * * * * * *
            REG     0000H     0008H     ABSOLUTE     "REG BANK 0"
            IDATA   0008H     0001H     UNIT         ?STACK

            * * * * * * *   C O D E   M E M O R Y   * * * * * * *
            CODE    0000H     0003H     ABSOLUTE     
            CODE    0003H     001FH     UNIT         ?PR?MAIN?MAIN
            CODE    0022H     0011H     UNIT         ?PR?INITIAL_IO?MAIN
            CODE    0033H     000CH     UNIT         ?C_C51STARTUP



OVERLAY MAP OF MODULE:   MA82G5Dxx (MAIN)


SEGMENT
  +--> CALLED SEGMENT
---------------------
?C_C51STARTUP
  +--> ?PR?MAIN?MAIN

?PR?MAIN?MAIN
  +--> ?PR?INITIAL_IO?MAIN



SYMBOL TABLE OF MODULE:  MA82G5Dxx (MAIN)

  VALUE           TYPE          NAME
  ----------------------------------

  -------         MODULE        MAIN
  C:0000H         SYMBOL        _ICE_DUMMY_
  D:0091H         PUBLIC        P1M0
  D:0095H         PUBLIC        P2M0
  D:0090H         PUBLIC        P1
  D:00B3H         PUBLIC        P4M0
  D:00A0H         PUBLIC        P2
  D:00C0H         PUBLIC        XICON
  D:00B0H         PUBLIC        P3
BL51 BANKED LINKER/LOCATER V6.00                                                      09/05/2017  17:55:54  PAGE 2


  D:00E8H         PUBLIC        P4
  D:00F8H         PUBLIC        P6
  D:00A8H         PUBLIC        IE
  D:00B8H         PUBLIC        IP0L
  D:00D8H         PUBLIC        CCON
  C:0003H         PUBLIC        main
  B:0090H.0       PUBLIC        P10
  B:00A0H.0       PUBLIC        P20
  B:00B0H.0       PUBLIC        P30
  B:00E8H.0       PUBLIC        P40
  D:0089H         PUBLIC        TMOD
  D:0088H         PUBLIC        TCON
  C:0022H         PUBLIC        Initial_IO
  B:0088H.7       PUBLIC        TF1
  D:008DH         PUBLIC        TH1
  D:008BH         PUBLIC        TL1
  B:0088H.6       PUBLIC        TR1
  D:0098H         PUBLIC        S0CON
  D:00C8H         PUBLIC        T2CON
  D:00D0H         PUBLIC        PSW
  -------         PROC          INITIAL_IO
  C:0022H         LINE#         9
  C:0022H         LINE#         10
  C:0022H         LINE#         11
  C:0025H         LINE#         12
  C:0027H         LINE#         13
  C:0029H         LINE#         15
  C:002CH         LINE#         16
  C:002FH         LINE#         17
  C:0032H         LINE#         18
  -------         ENDPROC       INITIAL_IO
  -------         PROC          MAIN
  C:0003H         LINE#         20
  C:0003H         LINE#         21
  C:0003H         LINE#         22
  C:0006H         LINE#         24
  C:0009H         LINE#         25
  C:000FH         LINE#         26
  C:0011H         LINE#         27
  C:0013H         LINE#         29
  C:0013H         LINE#         30
  C:0013H         LINE#         31
  C:0015H         LINE#         32
  C:0017H         LINE#         33
  C:0019H         LINE#         34
  C:001BH         LINE#         35
  C:001EH         LINE#         36
  C:0020H         LINE#         37
  -------         ENDPROC       MAIN
  -------         ENDMOD        MAIN

Program Size: data=9.0 xdata=0 code=63
LINK/LOCATE RUN COMPLETE.  0 WARNING(S),  0 ERROR(S)
